:020000040000FA
:0200000048288E
:080008008B13AB0083120313FC
:100010000B1813288C1E0D28342043202B088C121B
:100020000B108B170900851D1A20061E2120061FA4
:100030002B200D28A00A0A30031120020319A00169
:100040000800A00A0311A00303192828A003080030
:100050000930A00008000C1E2B28200899008316E8
:10006000981C3028831208008C1E34288C121A0821
:10007000A700A4012308A4002208A3002108A200CD
:100080002708A1000800A80B4328A90B4328080053
:1000900003179E019F010313831600308700503021
:1000A00086000830850083128B170B178B1583167B
:1000B0008C1683128C120B1003175030960003130A
:1000C00083160830960019309900181598161812E2
:1000D000831298171816A001A101A201A301A4017F
:1000E0000130AA00203084008316FF308500FF30E5
:1000F000870083120008972087002A08850083164E
:1001000000308700083085008312AA0D8E20840AF3
:10011000253003110402031992207428AA1D080037
:10012000AA0D0800203084000130AA0008008207D0
:100130003F3406345B344F3466346D347C340734DA
:060140007F346734080063
:02400E00D430AC
:00000001FF
